:100000000C94F00C0C94180D0C94180D0C94922078
:100010000C94180D0C94180D0C94180D0C94180DCC
:100020000C94180D0C94180D0C94180D0C94180DBC
:100030000C94180D0C94180D0C94180D0C94180DAC
:100040000C9448200C94180D0C94180D0C94180D59
:100050000C94180D0C9469210C94180D0C94180D27
:100060000C94180D0C94180D4465616374697661E5
:100070007465640053656C65637420546970004551
:100080006E74657220546970204E616D6500FFE0EA
:10009000FFD1AFFF32FFD0FFFEFFE0FFD1AEFFD0B8
:1000A000FFFEFFE0FFD11000FFFEFFD0FFE0FFC129
:1000B000FFD1AED580A83FD300408D142000A1C849
:1000C000DA1281CFD9F1DB402EA4A6AFFFD0FFFE1C
:1000D00000000000240027002A0000000000250086
:1000E00028002B0000000000230026002900040443
:1000F00004040404040402020202020203030303D0
:1001000003030102040810204080010204081020AB
:10011000010204081020506C6561736520776169E5
:10012000742E2E2E004144433A20200074656D70D9
:100130003A2000536574206D6561737572656400C3
:10014000537465703A200043616C6962726174692E
:100150006F6E002056005663633A20200020560040
:1001600056696E3A2000204300546D703A200046D4
:1001700069726D776172653A20003030300030303E
:100180003000560020484F4C440020484541540060
:10019000574F524B5900424F4F535400534C454513
:1001A000500020204F4646004552524F520000005A
:1001B0000008000201000003040700000000000026
:1001C000000000574DFBF12A000000002A3A002BE6
:1001D000F82A001717452507140082000383800FB3
:1001E00083E01FC7E00FC7E007C7C003EF8001EF40
:1001F0000000FE00F8FE3EFFFFFEFFFFFEFFFFFED9
:10020000FE7CFE80FE0201EF0003EF8007EFC007D7
:10021000C7C00FC7E01F83F00783C00183002323FB
:10022000AF3B0C000001E000000001E00000000115
:10023000E000000001E000000001E000000001E03B
:1002400000000001E000000001E000000001E0000B
:10025000000001E000000001E000000001E00000FB
:100260000001E000000001E000000001E0000000EB
:1002700001E00000FFFFFFFFE0FFFFFFFFE0FFFFE7
:10028000FFFFE0FFFFFFFFE00001E000000001E0F2
:1002900000000001E000000001E000000001E000BB
:1002A000000001E000000001E000000001E00000AB
:1002B0000001E000000001E000000001E00000009B
:1002C00001E000000001E000000001E0000000018A
:1002D000E000000C0F1E1203F80FF00FF00FE01FEC
:1002E000E01FC01FC03F803F803F007F007E007E38
:1002F000007C00FC00FC000F081013020BFFFEFF47
:10030000FEFFFEFFFEFFFEFFFEFFFEFFFE080808E9
:10031000120600FFFFFFFFFFFFFFFF132E8A1903E6
:10032000FD0007E00007E00007C0000FC0000FC09D
:10033000000F80001F80001F80001F80001F000032
:100340003F00003F00003E00007E00007E00007C79
:100350000000FC0000FC0000FC0000F80001F800B8
:1003600001F80001F00003F00003F00003F00007C3
:10037000E00007E00007E00007C0000FC0000FC06A
:10038000000F80001F80001F80001F80003F0000C2
:100390003F00003F00003E00007E00007E00007C29
:1003A0000000FC0000FC0000FC00001D2CB021023D
:1003B000FF001FC00000FFF80003FFFC0007FFFF65
:1003C000000FFFFF800FFFFF801FF0FFC03FC03F07
:1003D000C03FC03FE03F801FE07F801FF07F001FD5
:1003E000F07F000FF07F000FF0FF000FF0FF000F15
:1003F000F8FF000FF8FF000FF8FF000FF8FF000FE5
:10040000F8FF000FF8FF000FF8FF000FF8FF000FD4
:10041000F8FF000FF8FF000FF8FF000FF8FF000FC4
:10042000F8FF000FF87F000FF07F000FF07F000F44
:10043000F07F001FF07F801FF03F801FE03FC03F34
:10044000E03FC03FC01FF0FFC00FFFFF800FFFFF66
:100450000007FFFF0003FFFE0000FFF800001FC0C1
:1004600000122A7E210600003FC0007FC000FFC0AE
:1004700003FFC00FFFC03FFFC0FFFFC0FFFFC0FF73
:10048000FFC0FF3FC0FE3FC0F83FC0E03FC0003F9D
:10049000C0003FC0003FC0003FC0003FC0003FC0A1
:1004A000003FC0003FC0003FC0003FC0003FC00051
:1004B0003FC0003FC0003FC0003FC0003FC0003F02
:1004C000C0003FC0003FC0003FC0003FC0003FC071
:1004D000003FC0003FC0003FC0003FC0003FC00021
:1004E0003FC0003FC01D2BAC210200000FF00000F8
:1004F0007FFE0001FFFF0003FFFF8007FFFFC00F2B
:10050000FFFFE01FF83FF01FF01FF01FE00FF03F6C
:10051000C007F83FC007F83FC007F8000007F80021
:100520000007F800000FF800000FF000001FF000B7
:10053000001FF000003FE000007FE00000FFC0006F
:1005400001FF800003FF800007FF00000FFE000096
:100550001FFC00003FF800007FF00000FFE00001FA
:10056000FF800003FF00000FFE00001FFC00003FA3
:10057000F000007FE00000FFC00000FFFFFFF8FF79
:10058000FFFFF8FFFFFFF8FFFFFFF8FFFFFFF8FF97
:10059000FFFFF8FFFFFFF81C2CB02103FF007FC016
:1005A0000003FFF80007FFFC001FFFFF003FFFFFF5
:1005B000003FFFFF807FE0FFC07FC07FC0FF803F24
:1005C000C0FF001FE0FF001FE0FF001FE000001F52
:1005D000E000001FE000001FE000003FC000007FBF
:1005E000C00003FF80007FFF00007FFC00007FF061
:1005F00000007FF800007FFE00007FFF800000FF0A
:10060000C000003FE000001FE000001FE000000FFE
:10061000F000000FF000000FF0FF000FF0FF000FE0
:10062000F0FF000FF0FF001FE0FF801FE07FC03FE2
:10063000E07FE0FFC03FFFFF803FFFFF001FFFFEA6
:10064000000FFFFC0003FFF800007FC0001F2AA876
:100650002101000001FFC00001FFC00003FFC00036
:1006600007FFC00007FFC0000FFFC0000FFFC00062
:100670001FFFC0003FFFC0003FBFC0007F3FC00062
:10068000FF3FC000FE3FC001FE3FC001FC3FC00372
:10069000F83FC007F83FC007F03FC00FF03FC01F52
:1006A000E03FC01FC03FC03FC03FC03F803FC07F52
:1006B000803FC0FF003FC0FF003FC0FFFFFFFEFFC5
:1006C000FFFFFEFFFFFFFEFFFFFFFEFFFFFFFEFF3E
:1006D000FFFFFEFFFFFFFE00003FC000003FC00025
:1006E000003FC000003FC000003FC000003FC0000E
:1006F000003FC000003FC000003FC01D2BAC2102E6
:10070000FF7FFFFFE07FFFFFE07FFFFFE07FFFFF56
:10071000E07FFFFFE07FFFFFE07FFFFFE07F8000E3
:10072000007F8000007F8000007F8000007F8000CD
:10073000007F8000007F8000007F8000007F87F8BE
:10074000007F9FFE007FFFFF807FFFFFC07FFFFFD6
:10075000C07FFFFFE07FF03FF07FC01FF07F800F82
:10076000F07F800FF87F0007F8000007F80000070F
:10077000F8000007F8000007F8000007F80000077D
:10078000F0FF000FF0FF000FF0FF001FF0FF803FB1
:10079000E07FE0FFC07FFFFFC03FFFFF801FFFFF44
:1007A000000FFFFC0003FFF800007FC0001D2CB00D
:1007B0002102FF000FF000007FFC0000FFFF00039C
:1007C000FFFF8007FFFFC007FFFFE00FFC3FE01FB8
:1007D000F00FF01FE00FF03FC007F83FC007F83FF1
:1007E0008000007F8000007F8000007F8000007F0D
:1007F000000000FF03F800FF1FFE00FF3FFF00FFA7
:100800007FFF80FFFFFFC0FFFFFFE0FFF83FF0FF2B
:10081000E01FF0FFC00FF0FFC00FF8FF8007F8FFE8
:100820008007F8FF8007F8FF8007F8FF8007F87F50
:100830008007F87F8007F87F8007F07FC00FF03FC8
:10084000C00FF03FE01FE01FF83FE01FFFFFC00FA9
:10085000FFFF8007FFFF0003FFFE0000FFF800001E
:100860003FC0001C2AA8210300FFFFFFF0FFFFFF8D
:10087000F0FFFFFFF0FFFFFFF0FFFFFFF0FFFFFFC4
:10088000F0FFFFFFF000000FF000000FF000001F6E
:10089000F000001FE000003FE000003FC000007FCC
:1008A000C000007FC00000FF800000FF800001FF4B
:1008B000000001FF000001FE000003FE000003FE37
:1008C000000007FC000007FC00000FF800000FF814
:1008D00000001FF800001FF000001FF000003FE0C4
:1008E00000003FE000007FC000007FC00000FFC0AC
:1008F0000000FF800001FF800001FF000003FF00F7
:100900000003FF000003FE000007FE000007FC00DC
:10091000001D2CB02102FF003FF00001FFFE000788
:10092000FFFF800FFFFFC01FFFFFE03FFFFFF03F13
:10093000F87FF07FE01FF07FE01FF87FC00FF87FA7
:10094000C00FF87FC00FF87FC00FF87FC00FF83FCF
:10095000E01FF03FE01FF01FF87FE00FFFFFC00730
:10096000FFFF0001FFFC0000FFF80003FFFE000F87
:10097000FFFF801FFFFFC03FF03FE07FE01FE07FF1
:10098000C00FF07FC00FF0FF8007F8FF8007F8FF6F
:100990008007F8FF8007F8FF8007F8FF8007F8FF5F
:1009A000C00FF8FFC00FF87FE01FF07FF03FF07F2F
:1009B000FFFFE03FFFFFE01FFFFFC00FFFFF8003CF
:1009C000FFFE00007FF0001D2CB02102FF001FC0C1
:1009D0000000FFF80003FFFE0007FFFF000FFFFF0E
:1009E000801FFFFF803FE0FFC03FC03FE07F801FD0
:1009F000E07F801FE07F000FF0FF000FF0FF000F8F
:100A0000F0FF000FF0FF000FF8FF000FF8FF000FDE
:100A1000F8FF000FF8FF801FF87F801FF87FC03FAE
:100A2000F87FE0FFF83FFFFFF81FFFFFF81FFFF719
:100A3000F80FFFE7F803FFC7F800FE07F000000714
:100A4000F000000FF000000FF000000FF000000FAA
:100A5000E07F801FE07F801FE03F803FC03FC07F7E
:100A6000C03FE0FF801FFFFF800FFFFF0007FFFE7A
:100A70000003FFFC0001FFF000003FC000081D1D47
:100A8000130800FFFFFFFFFFFFFFFF000000000053
:100A90000000000000000000FFFFFFFFFFFFFFFF5E
:100AA00000121A00001803700390207F001A00182B
:100AB000000000000B0000FFFFFFFFFFFFFFFFFF34
:100AC000FF11103013010601C00001C00001C00079
:100AD00001C00001C00001C00001C000FFFF80FF95
:100AE000FF8001C00001C00001C00001C00001C0C2
:100AF0000001C00001C0000708080B03023E3E3E93
:100B00003E3EF0F0F00902040B010DFF80FF80056E
:100B100005050B0502F8F8F8F8F8FF11184813015D
:100B200002FFFF80FFFF80C00380C00380C00380FE
:100B3000C00380C00380C00380C00380C00380C0A6
:100B40000380C00380C00380C00380C00380C00353
:100B500080C00380C00380C00380C00380C00380C6
:100B6000FFFF80FFFF80FFFF80061818130702FCBD
:100B7000FC1C1C1C1C1C1C1C1C1C1C1C1C1C1C1CD5
:100B80001C1C1C1C1C1C1C111848130102FFFF809C
:100B9000FFFF8000038000038000038000038000CB
:100BA0000380000380000380000380000380FFFFB8
:100BB00080FFFF80C00000C00000C00000C0000037
:100BC000C00000C00000C00000C00000FFFF80FFA8
:100BD000FF80FFFF80111848130102FFFF80FFFF15
:100BE00080000380000380000380000380000380F6
:100BF0000003800003800003800003801FFF801F2C
:100C0000FF80000380000380000380000380000356
:100C100080000380000380000380FFFF80FFFF80CF
:100C2000FFFF80111848130102C00380C00380C079
:100C30000380C00380C00380C00380C00380C00362
:100C400080C00380C00380C00380FFFF80FFFF805F
:100C50000003800003800003800003800003800005
:100C600003800003800003800003800003800003F2
:100C700080111848130102FFFF80FFFF80C00000B1
:100C8000C00000C00000C00000C00000C00000C0E4
:100C90000000C00000C00000FFFF80FFFF800003D5
:100CA0008000038000038000038000038000038035
:100CB000000380000380FFFF80FFFF80FFFF8011A3
:100CC0001848130102FFFF80FFFF80C00000C00032
:100CD00000C00000C00000C00000C00000C0000054
:100CE000C00000C00000FFFF80FFFF80C00380C085
:100CF0000380C00380C00380C00380C00380C003A2
:100D000080C00380FFFF80FFFF80FFFF801018304E
:100D1000130202FFFFFFFF000700070007000700A4
:100D2000070007000700070007000700070007008B
:100D3000070007000700070007000700070007007B
:100D4000070007111848130102FFFF80FFFF80C052
:100D50000380C00380C00380C00380C00380C00341
:100D600080C00380C00380C00380FFFF80FFFF803E
:100D7000C00380C00380C00380C00380C00380C064
:100D80000380C00380C00380FFFF80FFFF80FFFF60
:100D900080111848130102FFFF80FFFF80C003800D
:100DA000C00380C00380C00380C00380C00380C034
:100DB0000380C00380C00380FFFF80FFFF8000032B
:100DC0008000038000038000038000038000038014
:100DD000000380000380FFFF80FFFF80FFFF80058E
:100DE00010100B0502F8F8F8F8F8000000000000F9
:100DF000F8F8F8F8F80710100B03023E3E3E3E3EAE
:100E00000000003E3E3E3E3EF0F0F0FFFFFFFFFFE1
:100E1000FFFFFFFFFFFFFFFFFFFFFFFFFFFFFFFFE2
:100E2000FFFFFFFFFFFFFFFFFFFFFFFFFFFFFFFFD2
:100E3000FFFFFFFFFFFFFFFFFFFFFFFFFFFFFFFFC2
:100E4000FFFFFFFFFFFFFFFFFFFFFFFFFFFFFF00B1
:100E5000090F00FD0A01E803D820FFFD0CFD0BFD82
:100E600000000009000C010B0B0904008080808049
:100E70008080800000808004030309030790909025
:100E80000608080901014848FC4848FC4848070B87
:100E90000B0901FF107C929050381412927C1007BD
:100EA0000A0A09010042A4A4481010244A4A8407EF
:100EB0000A0A09010060909090606294889462012F
:100EC0000303090407808080030C0C0903FF204002
:100ED00040808080808080404020030C0C0903FF0C
:100EE0008040402020202020204040800707070924
:100EF000010310925438549210070707090101109A
:100F00001010FE1010100205050904FDC0C040407D
:100F100080070101090104FE020202090400C0C0A9
:100F2000070A0A090100020404081010204040804A
:100F3000070A0A0901003844828282828282443888
:100F4000070A0A090100103050901010101010FE0E
:100F5000070A0A0901007C8282040810204080FEF2
:100F6000070A0A090100FE0204081C020202827C30
:100F7000070A0A090100040C14244484FE04040432
:100F8000070A0A090100FE8080BCC2020202827CBC
:100F9000070A0A0901003C408080BCC28282827C30
:100FA000070A0A090100FE020404080810102020A4
:100FB000070A0A09010038448244384482824438CE
:100FC000070A0A0901007C828282867A020204787A
:100FD000020707090400C0C0000000C0C0020A0ADE
:100FE0000904FDC0C0000000C0C0404080050A0ADE
:100FF00009020008102040808040201008070404E7
:10100000090102FE0000FE050A0A090200804020D4
:1010100010080810204080070A0A0901007C82821B
:1010200002040810100010070A0A0901007C8282DD
:101030009EA2A69A80807C070A0A09010010284413
:10104000828282FE828282070A0A090100F8848273
:1010500084F884828284F8070A0A0901007C82806D
:101060008080808080827C070A0A090100F88482DF
:10107000828282828284F8070A0A090100FE808047
:1010800080F880808080FE070A0A090100FE8080C7
:1010900080F88080808080070A0A0901007C8280B5
:1010A00080808E8282827C070A0A09010082828205
:1010B00082FE8282828282050A0A090200F82020CA
:1010C000202020202020F8080A0A0901001F04041B
:1010D00004040404048478070A0A0901008284884D
:1010E00090E0A090888482070A0A0901008080802D
:1010F000808080808080FE070A0A0901008282C603
:10110000AAAA9292828282070A0A0901008282C2F6
:10111000A2928A86828282070A0A0901007C828260
:101120008282828282827C070A0A090100FC828212
:1011300082FC8080808080070C0C0901FE7C82820A
:1011400082828282A2927C0806070A0A090100FCB8
:10115000828282FC9088848282070A0A0901007CCC
:10116000828280700C0282827C070A0A090100FEDA
:10117000101010101010101010070A0A0901008238
:1011800082828282828282827C070A0A090100822C
:10119000828244444428282810070A0A0901008250
:1011A00082828292929292AA44070A0A09010082DC
:1011B000824428101028448282070A0A090100820A
:1011C000824428101010101010070A0A090100FEAE
:1011D0000204081020408080FE040C0C0903FFF07C
:1011E00080808080808080808080F0070A0A0901EA
:1011F0000080404020101008040402040C0C090276
:10120000FFF010101010101010101010F007040450
:10121000090106102844820801010900FFFF0303A9
:10122000030903088040200707070901007C020228
:101230007E82867A070A0A090100808080BCC28209
:101240008282C2BC0707070901007C8280808082FD
:101250007C070A0A0901000202027A8682828286DB
:101260007A0707070901007C8282FE80807C070ADA
:101270000A0901001C22222020F820202020070A31
:101280000A0901FD7A84848478807C82827C070A42
:101290000A090100808080BCC28282828282050AA3
:1012A0000A090200600000E02020202020F8060D3E
:1012B0000D0901FD0C00001C040404040484848452
:1012C00078070A0A090100808080828CB0C0B08C47
:1012D00082050A0A090200E0202020202020202088
:1012E000F8070707090100EC929292929282070791
:1012F00007090100BCC282828282820707070901B6
:10130000007C82828282827C070A0A0901FDBCC2BB
:10131000828282C2BC808080070A0A0901FD7A8627
:10132000828282867A0202020707070901009C6214
:1013300042404040400707070901007C82807C0250
:10134000827C0709090901002020FC20202020229E
:101350001C0707070901008484848484847A0707B2
:101360000709010082824444282810070707090161
:10137000008282929292AA440707070901008244E0
:101380002810284482060A0A0901FD848484848482
:101390008C74048478070707090100FE04081020F4
:1013A00040FE050C0C0903FF3840404020C0C0201F
:1013B00040404038010C0C0904FF80808080808010
:1013C000808080808080050C0C0901FFE0101010E7
:1013D00020181820101010E007030309010762927B
:1013E0008CFFFFFFFFFFFFFFFFFFFFFFFFFFFFFF80
:1013F000FFFFFFFFFFFFFFFFFFFFFFFFFFFFFFFFFD
:10140000FFFF00000009000C010B0B0904008080A5
:101410000000808080808080800608080901000824
:10142000789490A0A47840070A0A0901001C2220A1
:1014300020F8202060A25C070606090103827C4494
:10144000447C82070A0A090100828244287C107CBD
:10145000101010010B0B0904FF8080808080008039
:1014600080808080040B0B0902FF60908060909068
:101470009060109060050202090209888808090935
:101480000900013C4299A5A1A599423C050707091D
:101490000103609070907800F807080809010112B4
:1014A00024489090482412060404090102FC040414
:1014B00004050101090204F80809090900013C4278
:1014C000B9A5B9A9A5423C060101090109FC04041A
:1014D00004090306609090600709090901011010D2
:1014E00010FE10101000FE040606090104609010A2
:1014F0006080F004060609010460902010906003EB
:1015000003030903082040800709090901FE8282BC
:10151000828282C6BA8080070A0A0901007E8A8A0E
:101520008A7A0A0A0A0A0A020202090404C0C004EA
:1015300003030902FD30906003060609010440C060
:10154000404040E00506060901047088887000F8F4
:101550000708080901019048241212244890070A3C
:101560000A09010040C0404042E60A121A06070A72
:101570000A09010040C040404CF2020C101E070A4C
:101580000A0901006090201092660A121A06070AE2
:101590000A0901001000101020408082827C070C94
:1015A0000C0901004020100038448282FE828282B1
:1015B000070C0C0901000408100038448282FE82E6
:1015C0008282070C0C0901001028440038448282F2
:1015D000FE828282070B0B090100629C0038448264
:1015E00082FE828282070B0B0901004444003844CA
:1015F0008282FE828282070B0B0901003844382860
:10160000448282FE828282070A0A0901006E90905B
:101610009090FC9090909E070D0D0901FD7C8280BA
:101620008080808080827C184830070C0C09010083
:1016300040201000FE404078404040FE070C0C095E
:10164000010004081000FE404078404040FE070CB6
:101650000C09010010284400FE404078404040FE44
:10166000070B0B090100444400FE40407840404015
:10167000FE050C0C09020080402000F820202020EC
:101680002020F8050C0C09020008102000F820208A
:1016900020202020F8050C0C09020020508800F8BA
:1016A000202020202020F8050B0B0902008888004C
:1016B000F8202020202020F8080A0A0900007C4297
:1016C0004141E1414141427C070B0B090100629C11
:1016D0000082C2A292928A8682070C0C0901004005
:1016E0002010007C8282828282827C070C0C09019D
:1016F00000040810007C8282828282827C070C0CAB
:10170000090100102844007C8282828282827C0748
:101710000B0B090100629C007C8282828282827CA7
:10172000070B0B0901004444007C82828282828282
:101730007C07070709010182442810284482070C0E
:101740000C0901FF027C868A8A9292A2A2C27C8046
:10175000070C0C09010040201000828282828282E4
:10176000827C070C0C09010004081000828282822E
:101770008282827C070C0C090100102844008282BE
:1017800082828282827C070B0B0901004444008222
:101790008282828282827C070C0C0901000408107C
:1017A000008282442810101010070A0A09010080E4
:1017B00080FC828282FC808080060A0A090100384F
:1017C000444448D04844444458070B0B09010020C6
:1017D0001008007C02027E82867A070B0B0901004A
:1017E000040810007C02027E82867A070B0B090136
:1017F00000102844007C02027E82867A070A0A09C9
:101800000100324C007C02027E82867A070A0A09B5
:1018100001004444007C02027E82867A070B0B0999
:101820000100182418007C02027E82867A070707CE
:101830000901006C92127C90926E070A0A0901FD60
:101840007C82808080827C184830070B0B09010065
:10185000402010007C8282FE80807C070B0B0901F7
:1018600000040810007C8282FE80807C070B0B093C
:101870000100102844007C8282FE80807C070A0AD6
:101880000901004444007C8282FE80807C050B0BB1
:1018900009020080402000E02020202020F8050BD5
:1018A0000B09020010204000E02020202020F80634
:1018B0000B0B090100205088007010101010107CD4
:1018C000050A0A090200909000E02020202020F85C
:1018D000070B0B090100483050087C82828282820B
:1018E0007C070A0A090100629C00BCC282828282D3
:1018F00082070B0B090100402010007C828282824B
:10190000827C070B0B090100040810007C82828294
:1019100082827C070B0B090100102844007C828224
:101920008282827C070A0A090100629C007C828212
:101930008282827C070A0A0901004444007C828278
:101940008282827C07090909010010381000FE001C
:101950001038100709090901FF027C8A8A92A2A2A5
:101960007C80070B0B0901004020100084848484D4
:1019700084847A070B0B0901000408100084848416
:101980008484847A070B0B090100102844008484A6
:10199000848484847A070A0A090100484800848400
:1019A000848484847A060E0E0901FD0810200084C8
:1019B000848484848C74048478070C0C0901FD8071
:1019C0008080BCC28282C2BC808080060D0D09016D
:1019D000FD48480084848484848C74048478A92914
:1019E00011241FBECFEFD8E0DEBFCDBF13E0A0E0D3
:1019F000B1E0E4EEFAE502C005900D92A23EB10717
:101A0000D9F725E0A2EEB3E001C01D92A432B207DF
:101A1000E1F71CE0C0EFDCE004C02197FE010E946A
:101A20006A2DCF3ED107C9F70E946A210C94702D10
:101A30000C9400004F925F926F927F928F929F92D0
:101A4000AF92BF92CF92DF92EF92FF920F931F93CC
:101A5000CF93DF9300D000D0CDB7DEB74B015C0150
:101A600029013A016701780120E030E0A9010E94D4
:101A7000842B87FDA6C020E030E0A901C301B2019C
:101A80000E94842B87FD9DC020E030E0A901C801A1
:101A9000B6010E94842B87FD94C081E02091C4048C
:101AA0003091C5042130310509F080E08093E504D0
:101AB0008092AA049092AB04A092AC04B092AD04C0
:101AC0004092AE045092AF046092B0047092B104A0
:101AD000C092B204D092B304E092B404F092B50480
:101AE0006091D8047091D9048091DA049091DB045C
:101AF0000E94312C20E030E04AE754E40E94892B18
:101B000069837A838B839C838092B6049092B70416
:101B1000A092B804B092B9049B01AC01C301B20118
:101B20000E94E82C2B013C014092BA045092BB0465
:101B30006092BC047092BD0429813A814B815C8122
:101B4000C701B6010E94892B6B017C01C092BE04C3
:101B5000D092BF04E092C004F092C1048091C2040C
:101B60009091C304019769F5A501940160E070E0CC
:101B7000CB010E94172B6093B6047093B704809337
:101B8000B8049093B904A301920160E070E0CB0126
:101B90000E94172B6093BA047093BB048093BC041B
:101BA0009093BD04A701960160E070E0CB010E9414
:101BB000172B6093BE047093BF048093C00490936E
:101BC000C1040F900F900F900F90DF91CF911F9154
:101BD0000F91FF90EF90DF90CF90BF90AF909F90CC
:101BE0008F907F906F905F904F90089580E0089560
:101BF0002091EE043091EF042817390799F1909362
:101C0000EF048093EE04009739F120910105FC0167
:101C1000211129C03596E491E09302050C96FC0150
:101C200084918093030580910205082E000C990B86
:101C300020910305821B910927FD939520910405AE
:101C4000203441F0829FC001112426E096958795AB
:101C50002A95E1F78093050586EF9DE090930005B6
:101C60008093FF040895213031F43F96E491E0938E
:101C700002054096D4CF3D96E491E09302050E967E
:101C8000CECFFC01808D8F5F0895AF92BF92CF922F
:101C9000DF92EF92FF920F931F93CF93DF936C012C
:101CA0007B018B01040F151FEB015E01AE18BF080D
:101CB000C017D10759F06991D601ED91FC910190BF
:101CC000F081E02DC6010995892B79F7C501DF91D7
:101CD000CF911F910F91FF90EF90DF90CF90BF9029
:101CE000AF900895833081F028F4813099F08230EC
:101CF000A9F008958730A9F08830C9F08430B1F494
:101D0000809180008F7D03C0809180008F778093C9
:101D10008000089584B58F7784BD089584B58F7D44
:101D2000FBCF8091B0008F778093B00008958091B1
:101D3000B0008F7DF9CFCF93DF93282F30E0F901EA
:101D4000E255FE4F8491F901EE5FFE4FD491F90107
:101D5000E251FF4FC491CC23A1F081110E94720E79
:101D6000EC2FF0E0EE0FFF1FEC51FF4FA591B49167
:101D7000EC91ED2381E090E009F480E0DF91CF91D8
:101D8000089580E090E0FACF1F93CF93DF93282F40
:101D900030E0F901E255FE4F8491F901EE5FFE4F0C
:101DA000D491F901E251FF4FC491CC23A9F0162F31
:101DB00081110E94720EEC2FF0E0EE0FFF1FE65231
:101DC000FF4FA591B4918FB7F894EC91111108C011
:101DD000D095DE23DC938FBFDF91CF911F910895C3
:101DE000DE2BF8CFCF93DF9390E0FC01EE5FFE4F48
:101DF000249182519F4FFC0184918823C9F090E087
:101E0000880F991FFC01E053FF4FA591B491FC018D
:101E1000E652FF4FC591D49161110DC09FB7F89460
:101E20008C91209582238C938881282328839FBFBF
:101E3000DF91CF910895623051F49FB7F8943C91AF
:101E4000822F809583238C93E8812E2BEFCF8FB741
:101E5000F894EC912E2B2C938FBFEACFCF93DF9386
:101E6000EC0161E089E00E94F20E209731F460E01D
:101E700089E0DF91CF910C94C40ECF3FD10511F4CE
:101E800061E0F6CFE7EBF1E0E491E33029F140F4D3
:101E9000E130B1F0E230D9F0C038D1058CF7E7CFAE
:101EA000E73021F1E83051F1E430B1F78091800062
:101EB000806280938000D0938B00C0938A0004C01E
:101EC00084B5806884BDC7BDDF91CF91089584B586
:101ED000806284BDC8BDF8CF809180008068809307
:101EE0008000D0938900C0938800EECF8091B0002D
:101EF00080688093B000C093B300E6CF8091B000BB
:101F000080628093B000C093B400DECF3FB7F894F6
:101F100080916C0490916D04A0916E04B0916F0457
:101F200026B5A89B05C02F3F19F00196A11DB11D34
:101F30003FBFBA2FA92F982F8827BC01CD01620F70
:101F4000711D811D911D42E0660F771F881F991F2B
:101F50004A95D1F708958F929F92AF92BF92CF92F8
:101F6000DF92EF92FF924B015C010E94860F6B01A2
:101F70007C010E94860F6C197D098E099F09683EBD
:101F8000734081059105A8F321E0821A9108A10808
:101F9000B10888EEC80E83E0D81EE11CF11C811444
:101FA0009104A104B10429F7FF90EF90DF90CF9046
:101FB000BF90AF909F908F9008952FB7F894609145
:101FC00068047091690480916A0490916B042FBF3A
:101FD00008950895DC011696ED91FC9117971296DD
:101FE0008C91481B477081E090E001C0880F4A95B2
:101FF000EAF7E60FF11D3081222319F0832B80834D
:10200000089580958323FBCFFB014181DC0112966B
:102010002C911297421768F013962C91139724175E
:1020200040F0608115962C91621718F424810C946D
:10203000EA0F0895FC0180819281980F928321819B
:10204000921760F494819F5F94839381890F821724
:1020500010F08FEF820F838381E0089580E0089570
:10206000FC01128280818150838314820895DB01F8
:10207000ED91FC9109940F931F93CF93DF931F92DF
:10208000CDB7DEB70091EC041091ED04E0911B0593
:10209000F0911C0582E0099530E020E04AE0B801AB
:1020A0008AEE94E00E943710182FE0911B05F09102
:1020B0001C0583E00995E0911B05F0911C0580E06B
:1020C00009951123B9F16091EC047091ED049E0122
:1020D0002F5F3F4F46E48AEE94E00E9437108981DB
:1020E0008093EA046091EC047091ED049E012F5FEF
:1020F0003F4F47E48AEE94E00E9437108981809335
:10210000EB046091EC047091ED0430E020E048E4D1
:102110008AEE94E00E9437108093F5046091EC04FD
:102120007091ED042DE135E047E18AEE94E00E94E4
:10213000371011E0812F0F90DF91CF911F910F91F8
:102140000895CF93DF9380912305811105C081E02D
:10215000809323050E943B10C091EC04D091ED04C4
:10216000E0911B05F0911C0582E00995E0911B05AB
:10217000F0911C0581E0099530E020E044E1BE01CA
:102180008AEE94E00E9437102DE135E047E1BE0170
:102190008AEE94E00E943710E0911B05F0911C0537
:1021A00080E0DF91CF9109940F931F93CF93E0913B
:1021B000F804F091F904309719F08AEE94E009954B
:1021C0000091EC041091ED04E0911B05F0911C05C9
:1021D00082E00995E0911B05F0911C0581E00995CD
:1021E00030E020E045E1B8018AEE94E00E9437102B
:1021F000C82F882341F02DE135E047E1B8018AEE90
:1022000094E00E943710E0911B05F0911C0580E0DE
:1022100009958C2FCF911F910F9108950B96FC017A
:10222000849108950A96FC0184910895FC0184919B
:1022300008950E941611882321F0823011F083E066
:10224000089586E00895FC01E60FF11D849190E069
:10225000982F88273196E4918E0F911D089568E09C
:102260000C94231166E00C9423115F926F927F927D
:102270008F929F92AF92BF92CF92DF92EF92FF9296
:102280000F931F93CF93DF93EC01E62EF42EC22E13
:102290000C811D81C8010E941611D82E8C819D8150
:1022A0000E941911982E21E0AA24AA94D21202C0E9
:1022B0002FE0A22E8C819D810E941211D82E8C813C
:1022C0009D810E940E11B82E8C819D810E942F113C
:1022D000E0E6EC1578F4009769F0080F191F91E615
:1022E000D92EBC14C0F4188A1B8A1C8A198A1A8A2F
:1022F00080E0A0C08C819D810E943211F0E4FC1529
:1023000038F4009729F0080F191F81E4D82EE9CF7F
:102310000F5E1F4FE6CFBD1430F3892D90E0F8011A
:1023200024912F3F31F40F5F1F4FBD14E1F2D3947E
:10233000F6CFCD1072C08C819D810E94161198013C
:102340002F5F3F4FF801882319F0823009F04EC00B
:1023500084918B8BF90124912C8BF8013396E491B5
:10236000E88BF8013496E491E98BF8013596E49115
:10237000EA8B0115110509F4BBCF8C819D810E9468
:1023800019113C89F31A9A89F91A9FEF930F9F0D3F
:102390002CA94EA94F1508F449C0921718F49F159F
:1023A00008F047C02B899989E90E9FEF920F9E0D87
:1023B0004BA95DA95E1508F44DC0941718F49E153D
:1023C00008F037C0080F111D295F722E769476949D
:1023D00076946F2C630E5E01FCE1AF0EB11C872C6E
:1023E000912CF61431F15E2C68014AC08491982F2B
:1023F0009F7092509A8B82958F70898BF9012491EE
:10240000822F8F708C8B22952F702B8BF801329638
:10241000E491E295EF70E88BACCF3296E491EA213B
:10242000E80FF92FF11D0E0F1F1F7FCF921708F035
:10243000B6CF8889DF91CF911F910F91FF90EF90D8
:10244000DF90CF90BF90AF909F908F907F906F90D4
:102450005F900895941708F0B2CFEBCFF601849106
:102460006A817B815C8EFD8E1F8E8E8F95014BE382
:10247000CE010E943710FFEFCF1ADF0A28E0520E7C
:102480008C2D801B871550F3080D191DF394A9CFCF
:10249000EF92FF920F931F93CF93DF93F82E062FA7
:1024A000E42E152FE091FF04F09100058AEE94E0F0
:1024B0000995080FCE2DD12F10E02991211108C0C8
:1024C000812FDF91CF911F910F91FF90EF90089591
:1024D000402F6F2D8AEE94E00E943511F80E180FF0
:1024E000ECCF0F931F93CF93DF938C01E091FF0408
:1024F000F09100058AEE94E00995D82FC0E0F8012C
:102500002491222351F04D2F6C2F8AEE94E00E94EB
:102510003511C80F0F5F1F4FF2CF8C2FDF91CF9176
:102520001F910F9108952EE93FE0009709F4089557
:10253000F9013197F1F70197F8CFCF93DF9300D0EE
:10254000CDB7DEB720ED37E03A8329839091BC0008
:10255000982311F081E00FC029813A81232B81F467
:102560008091A90481FDF6CF8091A80481110DC04E
:1025700091E09093A8040F900F90DF91CF91089570
:1025800029813A8121503109DFCF80E0F4CF84EAFC
:102590008093BC0061E080E80E949D12811102C01E
:1025A00080E008958091B900887F883051F08031B3
:1025B00041F08091A8048111F3CF82E08093A804B8
:1025C000EFCF88E78093BB0084E88093BC0062E093
:1025D00080E80E949D12882319F38091A90481FD4F
:1025E00005C08091B900887F883119F781E008958E
:1025F00084E98093BC0064E080E10C949D12809398
:10260000BB0084E88093BC0063E080E80E949D12D8
:102610008823A1F08091A90481FD0DC08091B900AB
:10262000887F883241F08091A804811106C092E031
:102630009093A804089581E0089580E00895109291
:10264000A80408958093A9041092B90084FF05C0DE
:102650008CE08093B8000C941F1388E4FACFCF93DA
:10266000DF93FC0123A5222389F0EC010E94C7120D
:10267000811104C080E0DF91CF9108958EA1811176
:1026800007C00E94FF128823A9F31BA681E0F3CFA5
:1026900080E4F7CF0F931F93CF93DF93C62FD42FF0
:1026A0008901633001F138F4613099F0623009F446
:1026B00049C0C1E012C0663029F1673091F1653040
:1026C000C1F70E942F13811117C00E94F812C0E0B9
:1026D00004C0FC0186A50E9422138C2FDF91CF91AC
:1026E0001F910F910895FC0116A221E023A741112B
:1026F000E0CF0E94F812DDCF8D2F0E94FF128111D2
:10270000D8CFE3CF0E942F138823F9F2DD2389F27B
:10271000F80181918F010E94FF128823B1F2D150FC
:10272000F5CF0E942F13882381F2DD2311F2F801E7
:1027300084910E94FF12C82F882379F20F5F1F4FE8
:10274000D150F3CFFC0146A321E023A7B2CFDB0198
:102750001496ED91FC9130E020E065E00994DB01F6
:102760001496ED91FC9130E020E062E00994DB01E9
:102770001496ED91FC9130E020E063E00994CF9253
:10278000DF92EF92FF920F931F93CF93DF938C0111
:102790007B016A0180E0F601C491811110C081E0E3
:1027A000CF3F49F04C2FB701C8010E94A7138823DF
:1027B00009F444C080E0BFEFCB1ADB0AECCF4FEF47
:1027C000CF3F89F3CE3FD9F1C03FA0F7C03E38F0EC
:1027D0004C2F4F70B701C8010E94AF13EBCFC03D23
:1027E00038F04C2F4F70B701C8010E94B713E2CFE9
:1027F000C03CF8F0D7011496ED91FC9130E020E058
:1028000040E064E0C8010995C295C07FCE5FD0E08A
:10281000CE010E949312D7011496ED91FC9130E005
:1028200020E041E064E0C8010995CE010E949312C6
:10283000C1CFC7FDBFCF8C2F90E0F8CF80E0DF91F4
:10284000CF911F910F91FF90EF90DF90CF9008955F
:10285000AF92BF92CF92DF92FF920F931F93CF93CD
:10286000DF936C018B01F42EE90180E1481709F434
:102870007EC0841778F1AAE04A1709F461C0BFE06E
:102880004B1709F47FC0F80102811381F2E3FF16B0
:1028900009F4DDC0FF1508F48EC085E1F81609F4CF
:1028A000DBC0A7E1FA1609F4ECC0B4E1FB1265C085
:1028B000D8011696ED91FC91179715968C918E0F75
:1028C0009F2F911D11928E179F07E1F7C8010E945B
:1028D000301053C0E1E14E1709F451C0F5E14F1338
:1028E000D2CFFB01A280B38042EA50E0C6010E9431
:1028F000BF13D50114964C91406BB801C6010E94DC
:10290000A71341E0B801C6010E94AF13F50126816B
:102910003781D8011496ED91FC91D50115964C9113
:1029200066E0C601099581111CC080E0DF91CF915E
:102930001F910F91FF90DF90CF90BF90AF900895BF
:10294000DB011496ED91FC9130E020E042E061E083
:10295000C60109954AEA50E0B801C6010E94BF13BA
:1029600092CF40E0B801C6010E94B7138CCF49E96D
:1029700050E0B801C6010E94BF1381E0D7CF4EE8F6
:1029800050E0F7CF41E0C6010E94B71340E0B80124
:10299000C6010E94AF1341E8B801C6010E94A71307
:1029A0004881B801C6010E94A71340E0B801C601E2
:1029B0000E94B713E2CFE6E4FE1609F46CC0F7E418
:1029C000FF1609F46DC08BE3F812D7CF99818B8184
:1029D00038E0390F813031F0833011F0392F02C0E7
:1029E000392F985021E0D80113964C91491708F4DB
:1029F00020E041E0391708F040E091E0F801528111
:102A0000351708F490E0322F342B932319F4242344
:102A100009F4B3CFFA80D12CC12C843048F490E073
:102A2000FC01EA5EFD4FC0808E5E9D4FDC01DC90B4
:102A3000F7FE04C0BE01C8010E94041088818C0DFD
:102A4000888389818D0D8983FF0C91F796CFBE0114
:102A5000C8010E94041091CFC8010E941A10882357
:102A600009F463CFD8011696ED91FC91179715964E
:102A70008C918E0F9F2F911D11928E179F07E1F75A
:102A80007CCF1882F80182818983858181508A8375
:102A900083818B8372CFD80115968C9188836DCFFB
:102AA000F8018181FBCF80917A00806980937A0060
:102AB0008EE480937C0061E070E080E090E00E9412
:102AC000AB0F83B7817F826083BF80E130E020E07D
:102AD00093B7916093BF889593B79E7F93BF909172
:102AE0007A0096FDFCCF4091780050917900240F38
:102AF000351F815069F780917A008F7780937A0033
:102B000084E0369527958A95E1F750E040E064EB44
:102B10007BE281E190E00E94BC2AC9010895809186
:102B20007A00806980937A0088EC80937C0064E16D
:102B300070E080E090E00E94AB0F83B7817F8260FD
:102B400083BF80E270E060E093B7916093BF8895A7
:102B500093B79E7F93BF90917A0096FDFCCF209112
:102B6000780030917900620F731F815069F780916E
:102B70007A008F7780937A0076956795769567953A
:102B800062527A4090E080E00E94312C26EF38E2D9
:102B90004CE151E40E94892B089590917A0090694C
:102BA00090937A008E50806480937C0083B7817FFD
:102BB000826083BF20E290E080E033B7316033BFB2
:102BC000889533B73E7F33BF30917A0036FDFCCF16
:102BD0004091780050917900840F951F215069F73A
:102BE00020917A002F7720937A0025E0969587959B
:102BF0002A95E1F708958FE00E94CD15A091770402
:102C0000B09178049C010E94082B0E94332C28E587
:102C100039E743E353E40E94892B0E94022CCB0145
:102C200008950F931F93CF938091B201882399F059
:102C3000CFEF0FEE11E061E085E00E94C40EC80105
:102C40000197F1F760E085E00E94C40EC80101978A
:102C5000F1F7C15081F7CF911F910F910895CF9255
:102C6000DF92EF92FF920F931F93CF93DF93D82EB3
:102C7000C92E86E00E949B0EC1E0892B09F0C0E0BE
:102C80000E94A11081E4E82E8EE0F82E8FE49EE0F1
:102C90000E94F80DF0920005E092FF040D2D1C2D0E
:102CA000D0E0F801419151918F016D2F80E00E9499
:102CB0004812D05FD038A9F70E94D4108111E6CF16
:102CC000CC2369F086E00E949B0EC1E0892B39F08D
:102CD0006AE070E080E090E00E94AB0FC0E086E028
:102CE0000E949B0E892B61F7C111ECCFDF91CF9130
:102CF0001F910F91FF90EF90DF90CF900C941116E1
:102D00005F926F927F928F929F92AF92BF92CF927B
:102D1000DF92EF92FF920F931F93CF93DF939090E8
:102D20009704AA24A394911001C0A12C80916C0156
:102D30008150990B10927E0410927D04880F991F88
:102D400090937C0480937B0481E090E090937A04DC
:102D500080937904892D90E0880F991F90938A04BD
:102D60008093890486E00E949B0EDD24D394892BF6
:102D700009F0D12C01E41EE046E0B42EC091890494
:102D8000D0918A04D595C795CC2E7E01FF24C7012A
:102D90008A0D911DA7FC9A9589199109A12C97FD7F
:102DA00006C08330910514F082E090E0A82E0E94C6
:102DB000A1108A2D0A2C000C990B3C012FEF621AEE
:102DC000720A629420EF62225C2C5A18E81AF90AFF
:102DD0008FE49EE00E94F80D109300050093FF041D
:102DE00084E790E00E9471124AE152E0662D80E093
:102DF0000E944812912C812C712C852D870D739483
:102E000090916C01891780F4C701880D991DB89EB7
:102E1000A001B99E500D11244B525E4F672D629553
:102E2000607F8CE00E9448128FEF881A980A23E096
:102E30007212E3CF0E94D4108111CACFDD2061F05D
:102E400086E00E949B0E892B39F06AE070E080E0FA
:102E500090E00E94AB0FD12C86E00E949B0E892B44
:102E6000B1F4D11014C00E941116C0929704DF91E2
:102E7000CF911F910F91FF90EF90DF90CF90BF9077
:102E8000AF909F908F907F906F905F9008959C2E51
:102E900075CF2F923F924F925F926F927F928F9257
:102EA0009F92AF92BF92CF92DF92EF92FF920F93D9
:102EB0001F93CF93DF9300D000D0CDB7DEB77C0156
:102EC000942EFC012080318077247394411101C03D
:102ED000712C70E0759567956A8310927E0410924C
:102EE0007D0462507109660F771F70937C046093B4
:102EF0007B0481E090E090937A0480937904892D9B
:102F000090E0880F991F90938A048093890486E04B
:102F10000E949B0E66246394892B09F0612CCC24BB
:102F2000CA944FE7D42E51E4A52E5EE0B52E8091D1
:102F3000890490918A04959587959C838B835B8007
:102F40008C011127C801870D911D77FC9A9589196D
:102F50009109712C97FD06C08330910514F082E031
:102F600090E0782E0E94A110272D072C000C330B27
:102F7000C9010196E82FE295E07FE9832C9DC0010D
:102F80002D9D900D3C9D900D1124080F191F000FD1
:102F9000111F8FE49EE00E94F80DB0920005A092F0
:102FA000FF04F7014081518160E080E00E944812F7
:102FB000FCE12F16F2E03F0661F44091970486E0B1
:102FC000489FA00111244B525E4F60E086E30E94AF
:102FD00048124AE152E0698180E00E944812882448
:102FE0008394912C412C4394852D840D87199A81CB
:102FF000891778F4F401EE0FFF1FE00FF11FEE0DBB
:10300000FF1D40815181642D6295607F8CE00E949C
:103010004812EFEF8E1A9E0AF3E04F12E4CF0E949F
:10302000D4108111B6CF662061F086E00E949B0E1D
:10303000892B39F06AE070E080E090E00E94AB0FED
:10304000612C86E00E949B0E892BE1F461101AC06E
:103050000E941116852D0F900F900F900F90DF9109
:10306000CF911F910F91FF90EF90DF90CF90BF9085
:10307000AF909F908F907F906F905F904F903F9018
:103080002F9008959B8053CF3F924F925F926F9203
:103090007F928F929F92AF92BF92CF92DF92EF92E8
:1030A000FF920F931F93CF93DF93CDB7DEB72E9789
:1030B0000FB6F894DEBF0FBECDBF8091A104882368
:1030C00009F4A5C11092A4041092A5041092A604BC
:1030D0001092A7048090A4049090A504A090A60448
:1030E000B090A704C0909204D0909304E090940410
:1030F000F0909504A7019601C501B4010E94172B19
:103100002B013C0120E030E0A9010E94E32C1816BD
:103110000CF0A0C1C301B2010E94022C80917F0477
:10312000882309F4B8C1C0926304D0926404E09289
:103130006504F0926604E12CF12C00EA10E420E032
:1031400030E040E450E46E31710540F0E12CF12CA8
:1031500000E81FE320E030E040E05FE360E070E083
:1031600080E391E40E941A0D8091E404882309F41D
:103170002AC10E94DD0F6D837E838F8398878091A3
:10318000CC049091CD04A091CE04B091CF044D8198
:103190005E816F817885481B590B6A0B7B0B809190
:1031A000D8049091D904A091DA04B091DB044817B7
:1031B00059076A077B0708F406C1E091C604F0913D
:1031C000C70480819181A281B38189839A83AB8373
:1031D000BC83E091CA04F091CB049C01AD016081F5
:1031E0007181828193810E94172B4B015C01209198
:1031F000D4043091D5044091D6045091D70469810C
:103200007A818B819C810E94172B6B017C0120911C
:10321000BA043091BB044091BC045091BD04C50177
:10322000B4010E94E82C2091D0043091D104409147
:10323000D2045091D3040E94182B2B013C014092E0
:10324000D0045092D1046092D2047092D304309092
:10325000E50431101AC02091B6043091B7044091B2
:10326000B8045091B904C701B6010E94E82C9B0133
:10327000AC01C301B2010E94172B6093D00470937C
:10328000D1048093D2049093D3044090D004509002
:10329000D1046090D2047090D3041091E004909116
:1032A000E1049E87A091E204AD870091E304212F01
:1032B000392F4A2F502FC301B2010E94E32C181658
:1032C0000CF0CCC0812F9E85AD85B02F8093D004AB
:1032D0009093D104A093D204B093D304332009F483
:1032E000D6C02091B6043091B7044091B8045091F3
:1032F000B904C501B4010E94E82C4B015C01209186
:10330000BE043091BF044091C0045091C104C70174
:10331000B6010E94E82C9B01AC016091D004709131
:10332000D1048091D2049091D3040E94172BA5015F
:1033300094010E94182B6B017C019B01AC01612F51
:103340007E858D85902F0E94842B87FD18C010915B
:10335000DC049091DD049E87A091DE04AD8700918E
:10336000DF04212F392F4A2F502FB601C7010E94A9
:10337000842B87FD04C01C2DDE86ED860F2DE09189
:10338000C804F091C904812F9E85AD85B02F80833C
:103390009183A283B38389819A81AB81BC8180931D
:1033A000D4049093D504A093D604B093D7048D8110
:1033B0009E81AF81B8858093CC049093CD04A09377
:1033C000CE04B093CF0460919B0470919C048091D3
:1033D0009D0490919E040E94FB2BCB012E960FB66C
:1033E000F894DEBF0FBECDBFDF91CF911F910F913B
:1033F000FF90EF90DF90CF90BF90AF909F908F9015
:103400007F906F905F904F903F900C942E0F809123
:10341000A004609184017091850181110EC080919A
:1034200090049091910420919F04BC01222329F0E3
:1034300060917F01680F792F711D90E080E00E94FC
:10344000312C6093A4047093A5048093A6049093F8
:10345000A70440CEC301B20190585ECE8091DC0437
:103460009091DD04A091DE04B091DF0489879A87F2
:10347000AB87BC879C01AD01C301B2010E94842BC4
:1034800087FF2CCF89859A85AB85BC851FCF812C82
:10349000912C540134CF20E030E040E05FE3C701DD
:1034A000B6010E94182B9B01AC01C501B4010E941A
:1034B000E32C18164CF410929B0410929C0410926A
:1034C0009D0410929E047FCF80E090E0AFE7B3E4CC
:1034D00080939B0490939C04A0939D04B0939E04BE
:1034E00072CF4F925F926F927F928F929F92AF9224
:1034F000BF92CF92DF92EF92FF92CF93DF938090B3
:10350000730490907404A0907504B0907604C091F8
:103510009704D0E0C501B4010E94FB2B6B017C0134
:1035200020E030E048E453E4C501B4010E94842B5C
:1035300093E0CC0FDD1F9A95E1F7C45DDE4F87FF66
:1035400031C02881398150E040E0255131094109DD
:103550005109C701B6010E945A2D28EC30E040E025
:1035600050E00E94BC2ACA01B9016B5E7F4F8F4FA9
:103570009F4F0E94332C6093920470939304809326
:10358000940490939504DF91CF91FF90EF90DF909A
:10359000CF90BF90AF909F908F907F906F905F90F3
:1035A0004F9008954A805B80712C612C20E030E0C0
:1035B0004CE853E4C501B4010E94842B87FF1FC06F
:1035C00088809980B12CA12CA7019601285C310933
:1035D00041095109C301B201681979098A099B0996
:1035E0000E945A2D20E530E040E050E00E94BC2AC5
:1035F000CA01B901680D791D8A1D9B1DBACF2C81A6
:103600003D8150E040E02419350946095709C701BA
:10361000B60168517140810991090E945A2D20E537
:1036200030E040E050E00E94BC2ACA01B901640DBC
:10363000751D861D971D9DCFDF92EF92FF920F9310
:103640001F93CF93DF93EC01D62E1CAD0BAD7C0105
:1036500084E0E80EF11CE98DFA8DC7010995412F30
:10366000480F2D2D602FC7010E9435119BAD890F8A
:103670008BAF81E090E0DF91CF911F910F91FF9090
:10368000EF90DF9008950F931F93CF93DF938C01FA
:10369000D0E0C0E0F801EC0FFD1F6491662341F01B
:1036A00086EE94E00E941C1B892B11F02196F2CF2C
:1036B000CE01DF91CF911F910F910895682F86EE73
:1036C00094E00C941C1B2F923F924F925F926F924A
:1036D0007F928F929F92AF92BF92CF92DF92EF92A2
:1036E000FF920F931F93CF93DF9300D01F92CDB71C
:1036F000DEB7412C1B821A820EE310E040ECE42E70
:10370000F12CCC24C394D12C60E2262E7EEB872EA4
:10371000912C8A81898386E00E949B0E3324339406
:10372000892B09F0312C10937E0400937D04F092D4
:103730007C04E0927B04D0927A04C0927904E2E89F
:10374000F0E0F0938A04E093890431E4A32E3EE094
:10375000B32E8091890490918A0495958795582E6F
:10376000FFE18F1342C010937E0400937D04F0921A
:103770007C04E0927B04D0927A04C0927904909207
:103780008A04809289049FE5592E0E94A1108FE43B
:103790009EE00E94F80DB0920005A092FF048FE712
:1037A00090E00E94711240922105F0E3F09322050F
:1037B0008EE50E945E1B1092210520922205712C3D
:1037C000612C8981681648F580919704F30196E091
:1037D000989FE00DF11D1124EB52FE4F80810E9455
:1037E0005E1BEFEF6E1A7E0AECCF80E65812CDCF4B
:1037F00010937E0400937D04F0927C04E0927B049D
:10380000D0927A04C0927904E0E4F0E0F0938A0464
:10381000E093890480E2582EB8CF4092210520928F
:103820002205852D0E945E1B0E94D4108111AFCF0E
:10383000332061F086E00E949B0E892B39F06AE00C
:1038400070E080E090E00E94AB0F312C86E00E9497
:103850009B0E892B09F07DCF31107BCFA090970470
:10386000F6E0FA9D50011124C5018B529E4F5C0178
:10387000EA81FB81E80FF91F50820E9411166AE06D
:1038800070E080E090E00E94AB0FEA81FB8131960E
:10389000FB83EA83F9E04F0E8DE248123ACFF5013F
:1038A00015820F900F900F90DF91CF911F910F9184
:1038B000FF90EF90DF90CF90BF90AF909F908F9050
:1038C0007F906F905F904F903F902F900895089554
:1038D00090E080E00895FC0101900020E9F7319725
:1038E000AF01481B590BBC0186EE94E00C94450EC9
:1038F0008F929F92AF92BF920F931F93CF93DF93BC
:10390000CDB7DEB7A1970FB6F894DEBF0FBECDBF1F
:1039100019A2423008F44AE08E010F5D1F4F842E39
:10392000912CB12CA12CA50194010E94E62AE62F2E
:10393000B901CA01EA30F4F4E05DD801EE938D01DB
:10394000232B242B252B79F790E080E0109719F09A
:10395000CD010E946B1CA1960FB6F894DEBF0FBE7E
:10396000CDBFDF91CF911F910F91BF90AF909F90EE
:103970008F900895E95CE1CF4F925F926F927F92B2
:103980008F929F92AF92BF92CF92DF92EF92FF926F
:103990000F931F93CF936B017C01742EAC019B019D
:1039A0000E94552D882399F081E292E0CF911F91DA
:1039B0000F91FF90EF90DF90CF90BF90AF909F90CE
:1039C0008F907F906F905F904F900C946B1C46018E
:1039D0005701E894B7F82FEF3FEF4FE75FE7C501D6
:1039E000B4010E94552D81110DC02FEF3FEF4FE71D
:1039F0005FE7C501B4010E94842B18161CF485E210
:103A000092E0D4CF2FEF3FEF4FE75FE4C701B6015D
:103A10000E94E32C18161CF489E292E0C7CF2FEF26
:103A20003FEF4FE75FECC701B6010E94842B87FD93
:103A3000F3CF20E030E0A901C701B6010E94842B3A
:103A400010E000E087FF08C08DE20E945E1B8C0141
:103A5000F7FAF094F7F8F094C0E060E070E080E0EE
:103A60009FE37C1641F020E030E040E251E40E9408
:103A7000892BCF5FF6CFA70196010E94182B2B014F
:103A80003C010E94022C4B015C014AE00E94781C20
:103A90007C01E00EF11ECC23B1F1C501B4010E94FE
:103AA000312C9B01AC01C301B2010E94172B4B01C9
:103AB0005C018EE20E945E1BE80EF91EC15018F1F7
:103AC00020E030E040E251E4C501B4010E94E82C5E
:103AD0002B013C010E94022C4B01B12CA12C4AE08D
:103AE000C501B4010E94781CE80EF91EC501B4019D
:103AF0000E94312C9B01AC01C301B2010E94172B23
:103B00004B015C01DBCFC701CF911F910F91FF905B
:103B1000EF90DF90CF90BF90AF909F908F907F906D
:103B20006F905F904F9008957F928F929F92AF9287
:103B3000BF92CF92DF92EF92FF920F931F93CF939A
:103B4000DF937C0186E00E949B0E11E0892B09F037
:103B500010E091E4C92E9EE0D92E00E22AE0722EF8
:103B6000C0918904D0918A04D595C7950E94A1106F
:103B70004E01B12CA12C8FE49EE00E94F80DD09252
:103B80000005C092FF04F7014081518160E080E0B0
:103B90000E94481210922105009322058AE192E0CA
:103BA0000E946B1C7092210500932205209779F5E5
:103BB00088E690E00E94431B0E94D4108111DBCF65
:103BC000112361F086E00E949B0E892B39F06AE098
:103BD00070E080E090E00E94AB0F10E086E00E9471
:103BE0009B0E892B09F0BCCF1111BACF0E94111680
:103BF000CE01DF91CF911F910F91FF90EF90DF9059
:103C0000CF90BF90AF909F908F907F9008954AE0A3
:103C1000C501B4010E94781C8DE292E00E946B1CE9
:103C2000F70182819381009739F20E946B1CC4CF07
:103C30001F93CF93DF93EC01162F0E94A62A18172B
:103C400039F0612FCE01DF91CF911F910C94AE2AF4
:103C5000DF91CF911F910895AF92BF92CF92DF92E3
:103C6000EF92FF920F931F93CF93DF9360918B019D
:103C700082E090E00E94181E60918A0183E090E04B
:103C80000E94181E6091850184E090E00E94181E39
:103C90006091840185E090E00E94181E60917F0190
:103CA00086E090E00E94181E6091D30187E090E0CA
:103CB0000E94181E6091D20188E090E00E94181EB8
:103CC0006091D10189E090E00E94181E60919A04F1
:103CD0008AE090E00E94181E60917F048BE090E0E3
:103CE0000E94181E6091B2018CE090E00E94181EA4
:103CF000609197048DE090E00E94181E60916C0125
:103D00008EE090E00E94181E8FE0E82EF12C10E06B
:103D100006E080916C011817B8F5109F600111241E
:103D2000D0E0C0E0FE01EC0DFD1DEB52FE4F6081C6
:103D3000C7018C0F9D1F0E94181E2196C630D10509
:103D400089F7670186E0C80ED11C88E0189FE00162
:103D50001124C45DDE4F8EE0E80EF11C69812296CD
:103D6000C6010E94181E560182E0A80EB11CFE0179
:103D700032976081C60101960E94181E6501AE143B
:103D8000BF0461F71F5FC5CFDF91CF911F910F91E6
:103D9000FF90EF90DF90CF90BF90AF9008958F92FB
:103DA0009F92AF92BF92CF92DF92EF92FF92CF930A
:103DB0008FEF90E00E942E0F83ED9EE00197F1F7C8
:103DC0008EE00E94CD15BC0190E080E00E94312C75
:103DD0004B015C018AE00E949B0E9091620498174F
:103DE00029F091E0909396048093620480910901F8
:103DF0009FEF980F90930901811106C00E94FB1557
:103E0000909399048093980460919B0470919C0412
:103E100080919D0490919E040E94FB2BCB010E94F7
:103E20002E0FC0907304D0907404E0907504F0904D
:103E30007604A7019601C501B4010E94172B2DEC51
:103E40003CEC4CE45DE30E94E82CA70196010E9443
:103E5000182B60937304709374048093750490938B
:103E600076040E94711A6091A2047091A30490E0FC
:103E700080E00E94312C4B015C01C090A404D090E2
:103E8000A504E090A604F090A704A70196010E9463
:103E9000842B811151C02091920430919304409160
:103EA000940450919504C501B4010E94172B4B0155
:103EB0005C0120E030E0A9010E94E32C181694F583
:103EC00020E030E040EA50E4C501B4010E94E32C58
:103ED000181694F16091A2047091A30490E080E020
:103EE0000E94312CA70196010E94172B4B015C0107
:103EF00020E030E0A9010E94E32C181664F520E0D0
:103F000030E040E85FE3C501B4010E94842B18163D
:103F100064F1C701B6010E94022C7093A304609360
:103F2000A20423C020E030E040EA50ECC501B40117
:103F30000E94842B87FFCECF6091920470919304EE
:103F400080919404909195040E94022C7093A30494
:103F50006093A204BFCF20E030E040E85FEBC501F2
:103F6000B4010E94E32C87FFD4CF6091900470913C
:103F7000910490E080E00E94312C209192043091D5
:103F8000930440919404509195040E94172B6B0167
:103F90007C0120E030E0A9010E94E32C18160CF00F
:103FA0006EC0C701B6010E94022C6530710508F091
:103FB0006AC080910502811105C08091D4018111F0
:103FC0000E94111681E0809305021092D401809125
:103FD000A2049091A304853F21E0920710F0109273
:103FE000080120910801211140C0843F9140E8F56B
:103FF0008FEF90E00E942E0F0E941116C1E0C09337
:1040000008010E9480160E942C1EC09396048EE028
:104010000E94CD15BC0190E080E00E94312C60939D
:1040200073047093740480937504909376041092D3
:10403000880480919004909191042CE231E03093B7
:104040007E0420937D0420E233E030937C042093AF
:104050007B042AE030E030937A0420937904880FBF
:10406000991F90938A0480938904CF91FF90EF90D9
:10407000DF90CF90BF90AF909F908F900895C70131
:10408000B601905890CF10920502A1CF0C94A62AA9
:104090001F920F920FB60F9211242F933F938F937D
:1040A0009F93AF93BF938091680490916904A0910E
:1040B0006A04B0916B043091670423E0230F2D371D
:1040C00058F50196A11DB11D2093670480936804E3
:1040D00090936904A0936A04B0936B0480916C047C
:1040E00090916D04A0916E04B0916F040196A11D92
:1040F000B11D80936C0490936D04A0936E04B093F3
:104100006F04BF91AF919F918F913F912F910F902D
:104110000FBE0F901F90189526E8230F0296A11D41
:10412000B11DD2CF1F920F920FB60F9211242F9371
:104130003F934F935F936F937F938F939F93EF93EF
:10414000FF9383B1817029B190917204981709F49B
:104150009DC030E0220F232F221F330B922F80931C
:10416000720440917104241709F490C020937104E3
:104170002091790430917A04981719F0319521959E
:1041800031094091890450918A0460917D047091B5
:104190007E04240F351F261737070CF48BC020919F
:1041A000790430917A04981719F0319521953109E5
:1041B0004091890450918A0460917B0470917C0441
:1041C000240F351F621773070CF46FC040917904F8
:1041D00050917A04981719F0519541955109209101
:1041E000890430918A04240F351F30938A04209368
:1041F000890441E0981340E020917004421709F4CB
:1042000040C02091790430917A04981719F03195C3
:10421000219531096091890470918A04E0917D04AF
:10422000F0917E04260F371F2E173F070CF44CC069
:104230002091790430917A04981719F031952195DD
:1042400031096091890470918A04E0917B04F091B6
:104250007C04260F371FE217F3078CF120917904B5
:1042600030917A04981719F0319521953109809190
:10427000890490918A04820F931F90938A048093FB
:1042800089044093700481E080939604FF91EF913C
:104290009F918F917F916F915F914F913F912F915E
:1042A0000F900FBE0F901F90189520917B043091B6
:1042B0007C049BCF20917D0430917E0496CF809129
:1042C0007B0490917C04D9CF80917D0490917E04F1
:1042D000D4CF1895CF93DF93CDB7DEB72D970FB618
:1042E000F894DEBF0FBECDBF789484B5826084BDE4
:1042F00084B5816084BD85B5826085BD85B58160EA
:1043000085BD80916E00816080936E001092810067
:104310008091810082608093810080918100816022
:1043200080938100809180008160809380008091E3
:10433000B10084608093B1008091B000816080936F
:10434000B00080917A00846080937A0080917A0036
:10435000826080937A0080917A00816080937A00F5
:1043600080917A00806880937A001092C10060E0AA
:104370008EE00E94F20E60E08FE00E94F20E61E09B
:1043800085E00E94F20E61E089E00E94F20E62E098
:1043900087E00E94F20E62E088E00E94F20E62E086
:1043A00086E00E94F20E62E08AE00E94F20E8FEF39
:1043B00090E00E942E0F60E085E00E94C40E809184
:1043C0007A00876080937A0080917A008860809379
:1043D0007A00789481E080936B00809368008BBBB7
:1043E0008091F504883209F0B6C08FEF80930A05FA
:1043F00090E080E00E944620182F81E090E00E942B
:104400004620912F8C36974E09F0B5C082E090E09F
:104410000E944620182F83E090E00E944620912FB2
:1044200090938B0180938A0184E090E00E94462063
:10443000182F85E090E00E944620912F90938501EF
:104440008093840186E090E00E94462080937F0163
:1044500087E090E00E9446208093D30188E090E0BE
:104460000E9446208093D20189E090E00E9446207D
:104470008093D1018AE090E00E94462080939A04C4
:104480008BE090E00E94462091E0811101C090E015
:1044900090937F048CE090E00E94462091E081118F
:1044A00001C090E09093B2018DE090E00E94462020
:1044B000809397048EE090E00E944620282E8093FF
:1044C0006C01FCE28F2EF1E09F2EA5EDAA2EA1E05B
:1044D000BA2EBFE0EB2EF12C312C231409F457C077
:1044E00010E000E0C701800F911F0E944620F501F7
:1044F000E00FF11F80830F5F1F4F0630110591F70A
:10450000670136E0C30ED11C6EE0E60EF11C3401EB
:10451000C6010E944620082F10E0102F0027D3016B
:104520000D931C932601B2E04B0E511CC60101965F
:104530000E944620082BF301019311933F01620171
:104540004E145F0429F73394F8E08F0E911C26E097
:10455000A20EB11CC2CF823011F483E047CF81306C
:1045600009F444CF803309F043CF8FEF80930A05DD
:1045700080930B053DCF67EE90E080E00E94181E0F
:104580006CE681E090E00E94181E0E942C1E0E94A2
:10459000531590937804809377040E94FB159093B1
:1045A00099048093980400918A0110918B011093D3
:1045B0009104009390048EE00E94CD15BC0190E020
:1045C00080E00E94312C6093730470937404809394
:1045D0007504909376040E948F150E94711A20E052
:1045E00030E040EA51E4609192047091930480912C
:1045F0009404909195040E94182B6B017C01B801E2
:1046000090E080E00E94312C9B01AC01C701B60113
:104610000E94842B87FF04C090E080E00E942E0F50
:104620001092DC041092DD041092DE041092DF047C
:10463000412C512C7FE7672E73E4772E4092E004E3
:104640005092E1046092E2047092E304A090C804E6
:10465000B090C9048091E404D501CD90DD90ED9037
:10466000FC90882309F449C6A3019201C701B60151
:104670000E94E32C181634F5F501408251826282C3
:1046800073828090D0049090D104A090D204B09016
:10469000D304C090E004D090E104E090E204F090F4
:1046A000E304A7019601C501B4010E94E32C18168A
:1046B000CCF4C092D004D092D104E092D204F09213
:1046C000D30420C020E030E0A901C701B6010E9458
:1046D000842B87FFD6CFD5011D921D921D921C926F
:1046E0001397CFCFC090DC04D090DD04E090DE04BF
:1046F000F090DF04A7019601C501B4010E94842B4C
:1047000087FDD7CF81E08093E40483B181708093EB
:10471000720489B190E0880F892F881F990B8093CC
:104720007104209172049091710481E0291380E05A
:10473000809370048CE291E090937E0480937D04DA
:1047400080E293E090937C0480937B048AE090E085
:1047500090937A0480937904000F111F10938A04B8
:10476000009389040E94DD0F60938C0470938D0484
:1047700080938E0490938F040E9411160E9411164C
:10478000E0918904F0918A04FA87E987F595E79525
:10479000FC87EB87F0939104E093900486E00E94FD
:1047A0009B0E8D8781119BC080918804882309F41A
:1047B00096C00E9411160E94DD0F6B017C01C09211
:1047C0008404D0928504E0928604F092870486E007
:1047D0000E949B0E892B59F40E94DD0F6C197D09F4
:1047E0008E099F09643F71408105910580F30E9405
:1047F000DD0F6C197D098E099F09643F71408105A9
:10480000910508F40DC58FEF90E00E942E0F0E94D5
:10481000111610E03AE0232E312C412F62E18FEB8C
:1048200091E00E944917182F8730A8F5E82FF0E093
:10483000E45EFB4D0C946A2D35246327E1274E2856
:104840005C286628742820E030E0A901C701B60181
:104850000E94842B87FF56CF1092D0041092D1046F
:104860001092D2041092D3044DCF90E2792E20E31F
:10487000622E412F6EE08DE691E00E944917182FBD
:10488000823009F4B1C208F059C1882309F482C109
:10489000813009F482C10E942C1E81E0809396042D
:1048A000AB85BC85B0939104A09390048CE291E019
:1048B00090937E0480937D0480E293E090937C0447
:1048C00080937B048AE090E090937A04809379044B
:1048D00089859A858E7F90938A0480938904BD850B
:1048E000B093880480919F04882309F11091D1012D
:1048F0001123E9F00E94DD0FC0908004D090810464
:10490000E0908204F09083046C197D098E099F0960
:1049100028EE33E040E050E00E94E62A211738F00C
:1049200010929F040E94111681E08093D40180911F
:1049300096048823E9F18091A004882349F120E0BE
:1049400030E040EA51E460919204709193048091C8
:104950009404909195040E94182B6B017C01609146
:1049600090047091910490E080E00E94312C9B01B2
:10497000AC01C701B6010E94842B87FF04C090E000
:1049800080E00E942E0F0E94111681E08093D401D6
:10499000109296041092A0041092A1040E94DD0FC0
:1049A00060938C0470938D0480938E0490938F0495
:1049B0000E94DD0F00918C0410918D0420918E04D3
:1049C00030918F04601B710B820B930B20E63AEE43
:1049D00040E050E00E94E62A122F20938B04809141
:1049E000A00481110BC08091D301882339F02817CE
:1049F00028F081E08093A0040E9411168091A10408
:104A000081110BC08091D201882339F0181728F04A
:104A100081E08093A1040E9411160E94CF1E0E9483
:104A200044180E94A11001E41EE088E2D82E93E50C
:104A3000F92E2FE0C22E34E1B32E44E3E42E56E0EB
:104A4000A52E65E2962E76E1872E8FE49EE00E94E9
:104A5000F80D109300050093FF044AE352E060E074
:104A600080E00E944812D0922105109222056091A8
:104A7000A4047091A5048091A6049091A70440E03D
:104A80000E94BC1CF0922105109222058091A20484
:104A90009091A304853F914008F4D8C388EA91E03F
:104AA0000E94431B80919A04882309F401C46091F9
:104AB00098047091990490E080E00E94312C20E0ED
:104AC00030E04AE754E40E94892B2B013C0110920C
:104AD0002105E0922205809197048A9DC00111244E
:104AE0008B529E4F0E946B1CF0922105E092220592
:104AF00041E0C301B2010E94BC1C82E891E00E9427
:104B0000431B80EA9AE00E94F80D10930005009381
:104B1000FF0490922105809222056091A204709179
:104B2000A3048EE791E0653FF1E07F0708F0D7C36B
:104B300090E080E04AE00E94781CD3C3833009F4FF
:104B400056C1843009F0A7CE80916C01883008F0FE
:104B5000B7C191E0980F90936C01809397040E94E5
:104B6000631BE0919704B8E0EB9FF0011124E45D32
:104B7000FE4F28ED30E03183208384E391E093837E
:104B80008283A6E8B1E0B583A4832EE130E03783C9
:104B900026836FCE0E9480166CCECE0101962C012A
:104BA000C12CD12C7601C39481E4282E8EE0382EBE
:104BB000E091970494E0E99FF0011124C601019768
:104BC000E80FF91FEE0FFF1FE45DFE4F808191811A
:104BD0009093910480939004A8ECB0E0B0937E048D
:104BE000A0937D04E8EEF3E0F0937C04E0937B0473
:104BF00021E030E030937A0420937904880F991FE4
:104C000090938A048093890431E03093D40186E044
:104C10000E949B0E01E0892B09F000E00E94CF1E4C
:104C20000E9444180E94A1108FE49EE00E94F80D9B
:104C3000309200052092FF0487E491E00E947112F7
:104C40001092210560E16093220580E491E00E94CA
:104C5000431B4AE0C701B6010E94781C8FE292E034
:104C60000E946B1C80910502109221057092220512
:104C7000882309F49DC083E391E00E94431B1092B6
:104C80002105609222058CE291E00E94431B8091F5
:104C9000890490918A04959587954C01092E000C02
:104CA000AA08BB0897FF80C08DE20E945E1B6627A2
:104CB0007727CB01681979098A099B094AE00E9484
:104CC000781C0E94D4108111AFCF002361F086E0E0
:104CD0000E949B0E892B39F06AE070E080E090E042
:104CE0000E94AB0F00E086E00E949B0E892B09F02A
:104CF00095CF011193CF8091890490918A04959565
:104D00008795D2018D939D932D010E9411166AE023
:104D100070E080E090E00E94AB0FBFEFCB1ADB0A9F
:104D2000EB0AFB0AE4E0CE16D104E104F10409F039
:104D30003FCF8FEF90E00E942E0F83ED9EE0019712
:104D4000F1F70E948F150E94022C1B0178876F8358
:104D5000A980BA80EB80FC80C5010A968E159F055C
:104D600008F087CDCD80DE80C7010A968C159D05A1
:104D700008F07FCD40E066E080E191E00E944917B5
:104D8000882309F476CDE091970428E0E29FF001B2
:104D90001124E45DFE4FB182A082F382E282D582CB
:104DA000C4823782268265CD4AE0C501B40187CF2F
:104DB00085E291E00E94431B60917304709174043A
:104DC00080917504909176040E94022C90E080E01E
:104DD0004AE00E94781C109221056092220586E12B
:104DE00091E00E94431B6DCF0E94631B42CD8091D6
:104DF0006C01813029F486E191E00E942F1639CDB3
:104E000040E066E08EE191E00E944917882309F4B2
:104E100030CD8091970490916C01A92FA150BB0BCC
:104E2000AD0106E08A171B0639F481508093970480
:104E3000915090936C011DCDE82FF0E0E417F50739
:104E4000BCF7809F7001112430E020E05F01BFEFCC
:104E5000AB1ABB0AB9016E0D7F1D6B527E4FDB0191
:104E60001696DC901697DC922F5F3F4F2630310567
:104E700089F7D50123E0AA0FBB1F2A95E1F7A45DAE
:104E8000BE4F2D913C91119763E0EE0FFF1F6A9585
:104E9000E1F7E45DFE4F3183208312962D913C9122
:104EA00013973383228314962D913C911597358364
:104EB000248316962D913C91378326838F5FBCCF38
:104EC00084E291E09ACF00E048E2442E512C50E970
:104ED000652E772473946CE2862E9924939470E265
:104EE000A72E73E0B72EE4E1CE2ED12CF8ECEF2EF6
:104EF000F12C402F6AE08CE891E00E944917082FBE
:104F0000813009F43FC0F8F0823009F086CC8091FE
:104F10007F0190E0D0927E04C0927D04F0927C04E8
:104F2000E0927B0430927A0420927904880F991FD2
:104F300090938A04809389048BE791E00E94941DEA
:104F400080937F01D6CF80918A0190918B019092BE
:104F50007E0480927D04B0927C04A0927B04309207
:104F60007A0420927904880F991F90938A04809381
:104F7000890486E891E00E94941D90938B018093B0
:104F80008A01B7CF809184019091850150927E046F
:104F900040927D0470927C0460927B0430927A048B
:104FA00020927904880F991F90938A048093890432
:104FB00080E891E00E94941D909385018093840184
:104FC00098CF00E0402F6AE082EA91E00E94491702
:104FD000082F813009F442C008F1823009F01DCC5D
:104FE0008091D10190E010927E0410927D04E8E659
:104FF000F1E0F0937C04E0937B0430927A042092F9
:105000007904880F991F90938A048093890486E914
:1050100091E00E94941D8093D101D4CF8091D3015F
:1050200090E010927E0410927D04ACE3B0E0B09367
:105030007C04A0937B04E1E0F0E0F0937A04E09339
:105040007904880F991F90938A04809389048EE9CC
:1050500091E00E94941D8093D301B4CF8091D2013E
:1050600090E010927E0410927D0428E730E03093A7
:105070007C0420937B04A5E0B0E0B0937A04A09375
:105080007904880F991F90938A04809389048AE990
:1050900091E00E94941D8093D20194CF40917F04AF
:1050A00066E089EB91E00E94491791E0811101C00F
:1050B00090E090937F04B1CB40919A0466E083EB3B
:1050C00091E00E94491780939A04A7CB4091B201C6
:1050D00066E08CEA91E00E94491791E0811101C0DD
:1050E00090E09093B20199CB86E00E949B0E01E084
:1050F000892B09F000E00E94531590937804809367
:105100007704BC0190E080E00E94312C20E030E088
:105110004AE754E40E94892B6B017C010E94FB1535
:105120009093990480939804BC0190E080E00E94E1
:10513000312C20E030E04AE754E40E94892B4B01F7
:105140005C010E948F152B013C010E94A1108FE48D
:105150009EE00E94F80D21E43EE03093000520938C
:10516000FF0410922105109222058FE691E00E9423
:10517000431B85E392E00E946B1C1092210530E1F5
:105180003093220589E691E00E94431B41E0C30170
:10519000B2010E94BC1C86E691E00E94431B109263
:1051A000210560E26093220580E691E00E94431BA6
:1051B00041E0C501B4010E94BC1C8DE591E00E9454
:1051C000431B1092210580E38093220586E591E040
:1051D0000E94431B41E0C701B6010E94BC1C83E54D
:1051E00091E00E94431B0E94D4108111B0CF002394
:1051F00061F086E00E949B0E892B39F06AE070E036
:1052000080E090E00E94AB0F00E086E00E949B0EE1
:10521000892B09F070CF01116ECF0E941116FDCAC3
:1052200080919F0491E0892780939F04882351F007
:105230000E94DD0F60938004709381048093820448
:105240009093830481E08093960449CB8091A104DC
:10525000882319F082EA91E023CC8091A00488236E
:1052600019F08CE991E01CCC80919F04882319F0FF
:1052700086E991E015CC80910502882319F080E938
:1052800091E00ECC20E030E044E353E460919B04D5
:1052900070919C0480919D0490919E040E94842BA7
:1052A00087FF03C08AE891E0FBCB84E891E0F8CB6C
:1052B00082EC91E00E94F80D109300050093FF042A
:1052C000C0922105B09222056091A2047091A304BE
:1052D000653F21E0720708F42BCC8AE791E00E9439
:1052E000431B0E94D4108111B0CB80E090E0892B49
:1052F00009F446CA0E94000043CAC092D004D0926A
:10530000D104E092D204F092D304E091C604F0916B
:10531000C70480819181A281B3818093D40490934A
:10532000D504A093D604B093D70420E030E04FE733
:1053300053E4C701B6010E94E32C18160CF083CA8F
:105340004092D0045092D1046092D2047092D3045F
:10535000D9C90F931F93CF938BE994E09093C9041D
:105360008093C80483E694E09093C7048093C604B6
:1053700084EA94E09093CB048093CA041092E404EE
:105380001092DC041092DD041092DE041092DF040F
:1053900080E090E0AFE7B3E48093E0049093E10411
:1053A000A093E204B093E30484E690E0A0E0B0E0D0
:1053B0008093D8049093D904A093DA04B093DB04CB
:1053C00081E090E09093C3048093C2049093C5045D
:1053D0008093C404C1E0C093E50480E090E0A0E3C2
:1053E000B1E48093AA049093AB04A093AC04B0936F
:1053F000AD0480E090E0A0E0BFE38093AE04909322
:10540000AF04A093B004B093B10480E090E0A0E8B2
:10541000BFE38093B2049093B304A093B404B09319
:10542000B50480E090E0A0E3B1EC8093B6049093E3
:10543000B704A093B804B093B9048DEC9CECACE431
:10544000BDEB8093BA049093BB04A093BC04B093CB
:10545000BD0480E090E0A0E2B1EC8093BE049093A4
:10546000BF04A093C004B093C1040E94DD0F00915B
:10547000D8041091D9042091DA043091DB04601B28
:10548000710B820B930B6093CC047093CD048093CB
:10549000CE049093CF041092E9041092E8048AE0BD
:1054A00092E09093E7048093E60410922105109215
:1054B0002205109223051092EF041092EE04109230
:1054C000F1041092F0041092F304C093F20482E20B
:1054D0008093F4041092F9041092F804EDE0F5E0E2
:1054E0008BE195E02FEF21938E179F07E1F781E085
:1054F00080930A0526EF3DE0309300052093FF04DA
:1055000080930105109202051092030580E48093B8
:1055100004051092050589EE9FE090931C05809389
:105520001B058AE091E09093ED048093EC0482E106
:10553000809318050E943B108AE092E09093E70464
:105540008093E604CF911F910F910895F999FECFB2
:1055500092BD81BDF89A992780B50895262FF999B3
:10556000FECF1FBA92BD81BD20BD0FB6F894FA9A46
:10557000F99A0FBE01960895052E97FB1EF400942C
:105580000E94D32A57FD07D00E94E62A07FC03D0C9
:105590004EF40C94D32A50954095309521953F4F69
:1055A0004F4F5F4F089590958095709561957F4F0F
:1055B0008F4F9F4F08950E94082BA59F900DB49F79
:1055C000900DA49F800D911D11240895A1E21A2E23
:1055D000AA1BBB1BFD010DC0AA1FBB1FEE1FFF1F97
:1055E000A217B307E407F50720F0A21BB30BE40BE7
:1055F000F50B661F771F881F991F1A9469F760952E
:105600007095809590959B01AC01BD01CF010895E7
:10561000A29FB001B39FC001A39F700D811D1124F3
:10562000911DB29F700D811D1124911D0895505838
:10563000BB27AA270E942F2B0C94A92C0E949B2CDD
:1056400038F00E94A22C20F039F49F3F19F426F480
:105650000C94982C0EF4E095E7FB0C94922CE92F17
:105660000E94BA2C58F3BA1762077307840795078C
:1056700020F079F4A6F50C94DC2C0EF4E0950B2EBA
:10568000BA2FA02D0B01B90190010C01CA01A00194
:105690001124FF27591B99F0593F50F4503E68F1EF
:1056A0001A16F040A22F232F342F4427585FF3CF30
:1056B000469537952795A795F0405395C9F77EF401
:1056C0001F16BA0B620B730B840BBAF09150A1F04A
:1056D000FF0FBB1F661F771F881FC2F70EC0BA0FD0
:1056E000621F731F841F48F4879577956795B79558
:1056F000F7959E3F08F0B0CF9395880F08F0992753
:10570000EE0F9795879508950E946E2C08F481E01E
:1057100008950E949D2B0C94A92C0E94A22C58F055
:105720000E949B2C40F029F45F3F29F00C94922CAE
:1057300051110C94DD2C0C94982C0E94BA2C68F317
:105740009923B1F3552391F3951B550BBB27AA273A
:1057500062177307840738F09F5F5F4F220F331F74
:10576000441FAA1FA9F335D00E2E3AF0E0E832D03C
:1057700091505040E695001CCAF72BD0FE2F29D03F
:10578000660F771F881FBB1F261737074807AB0711
:10579000B0E809F0BB0B802DBF01FF2793585F4F86
:1057A0003AF09E3F510578F00C94922C0C94DD2C2D
:1057B0005F3FE4F3983ED4F3869577956795B79568
:1057C000F7959F5FC9F7880F911D9695879597F973
:1057D0000895E1E0660F771F881FBB1F62177307EC
:1057E0008407BA0720F0621B730B840BBA0BEE1F01
:1057F00088F7E09508950E94022C6894B1110C94EA
:10580000DD2C08950E94C22C88F09F5798F0B92F84
:105810009927B751B0F0E1F0660F771F881F991FE5
:105820001AF0BA95C9F714C0B13091F00E94DC2C7F
:10583000B1E008950C94DC2C672F782F8827B85F8F
:1058400039F0B93FCCF3869577956795B395D9F73D
:105850003EF490958095709561957F4F8F4F9F4F47
:105860000895E89409C097FB3EF490958095709553
:1058700061957F4F8F4F9F4F9923A9F0F92F96E99C
:10588000BB279395F695879577956795B795F11111
:10589000F8CFFAF4BB0F11F460FF1BC06F5F7F4FAE
:1058A0008F4F9F4F16C0882311F096E911C07723C0
:1058B00021F09EE8872F762F05C0662371F096E8C9
:1058C000862F70E060E02AF09A95660F771F881F98
:1058D000DAF7880F9695879597F90895990F00083C
:1058E000550FAA0BE0E8FEEF16161706E807F907B2
:1058F000C0F012161306E407F50798F0621B730B4D
:10590000840B950B39F40A2661F0232B242B252BCD
:1059100021F408950A2609F4A140A6958FEF811D70
:10592000811D089597F99F6780E870E060E0089511
:105930009FEF80EC089500240A94161617061806A7
:105940000906089500240A94121613061406050683
:105950000895092E0394000C11F4882352F0BB0F14
:1059600040F4BF2B11F460FF04C06F5F7F4F8F4F77
:105970009F4F089557FD9058440F551F59F05F3FB2
:1059800071F04795880F97FB991F61F09F3F79F061
:1059900087950895121613061406551FF2CF4695E3
:1059A000F1DF08C0161617061806991FF1CF869565
:1059B0007105610508940895E894BB276627772749
:1059C000CB0197F908950E946E2C08F48FEF08958B
:1059D0000E94FB2C0C94A92C0E949B2C38F00E9456
:1059E000A22C20F0952311F00C94922C0C94982C5E
:1059F00011240C94DD2C0E94BA2C70F3959FC1F3F6
:105A0000950F50E0551F629FF001729FBB27F00D6C
:105A1000B11D639FAA27F00DB11DAA1F649F6627C1
:105A2000B00DA11D661F829F2227B00DA11D621F10
:105A3000739FB00DA11D621F839FA00D611D221FCA
:105A4000749F3327A00D611D231F849F600D211DAE
:105A5000822F762F6A2F11249F5750409AF0F1F031
:105A600088234AF0EE0FFF1FBB1F661F771F881F9A
:105A700091505040A9F79E3F510580F00C94922C14
:105A80000C94DD2C5F3FE4F3983ED4F38695779534
:105A90006795B795F795E7959F5FC1F7FE2B880F40
:105AA000911D9695879597F908950E946E2C880B05
:105AB000990B0895DB018F939F930E94DB2ABF917E
:105AC000AF91A29F800D911DA39F900DB29F900D4D
:105AD00011240895EE0FFF1F0590F491E02D099415
:045AE000F894FFCF68
:105AE400084000000080E20301FF281400014A136B
:105AF4003F025002530257025F026A02760280029A
:105B04005002530257028F029B02AA02D8003401AA
:105B140086011E00000000000000000000000000DC
:105B24000000000000000000000000000000000071
:105B34000000000000000000000000000000000061
:105B4400000000000000000000000000011C02B37F
:105B540002BE02CC02D702E202EE02F502000332D8
:105B64000603000396001103000340011E03110302
:105B74000603F502EE022C03380340034A035203E2
:105B84004A035E03520340032C03EE026D037403C5
:105B94007C030183038F039B03A603B303BA03BEF1
:105BA40003C9031E035E03A60383036D03D603EE3A
:105BB40002280F05014243312E3500000000000089
:105BC40000000000000000000000000000000000D1
:105BD40000000000000000000000000000000000C1
:105BE400000000000001000000001C1B450E681CA2
:105BF400671C000100FF0100FF003E005469703A79
:105C0400006E616E00696E66006F7666002000208B
:105C14006F6620330076312E38005345543A0053D2
:105C2400746F72652053657474696E6773203F00E6
:105C34004E6F00596573005761726E696E67005943
:105C44006F752063616E6E6F740064656C65746556
:105C540020796F7572006C6173742074697021000F
:105C640041726520796F752073757265203F005904
:105C74006F752072656163686564006D6178696D34
:105C8400756D206E756D626572006F662074697043
:105C94007321004368616E67652054697000436135
:105CA4006C696272617465205469700052656E613A
:105CB4006D65205469700044656C65746520546991
:105CC4007000416464206E657720546970005265E9
:105CD4007475726E00426F6F73742054656D70003A
:105CE400646567204300536C6565702054656D706E
:105CF4000044656661756C742054656D700054656C
:105D04006D702053657474696E677300426F6F73AE
:105D1400742054696D6572005365636F6E6473001B
:105D24004F66662054696D6572004D696E757465C1
:105D34007300536C6565702054696D657200546915
:105D44006D65722053657474696E67730042757A69
:105D54007A65720044697361626C6500456E6162C4
:105D64006C65004D61696E2053637265656E004217
:105D74006967204E756D62657273004D6F726520A0
:105D8400496E666F7300436F6E74726F6C20547942
:105D9400706500446972656374005049440053653A
:105DA400747570204D656E75005469702053657468
:105DB40074696E677300496E666F726D6174696FA2
:025DC4006E006F
:00000001FF
